:020000040800F2
:100000000080002095550008490B00084B0B0008A4
:100010004D0B00084F0B0008510B000800000000BA
:10002000000000000000000000000000530B00086A
:10003000550B000800000000570B0008590B000882
:10004000E5550008E5550008E5550008E5550008A8
:10005000E5550008E5550008E5550008E555000898
:10006000E5550008E5550008E5550008E555000888
:10007000610B0008710B0008810B0008E5550008B2
:10008000E555000800000000910B0008E555000848
:10009000E5550008E5550008E5550008E555000858
:1000A000E5550008E5550008E5550008E555000848
:1000B000A90B0008F10B0008E5550008E5550008FC
:1000C000E5550008E5550008E5550008E555000828
:1000D000E5550008090C0008E5550008E55500083D
:1000E000E5550008E5550008E5550008E555000808
:1000F000E5550008E5550008E5550008000000003A
:1001000000000000E555000800000000E55500086B
:10011000E555000800000000E5550008E555000819
:10012000E5550008E5550008E5550008E5550008C7
:10013000E55500080000000000000000E55500083B
:10014000E5550008E555000800000000000000002B
:10015000000000000000000000000000000000009F
:10016000000000000000000000000000E55500084D
:10017000E55500080000000000000000000000003D
:1001800000000000E555000800000000000000002D
:10019000000000000000000000000000000000005F
:1001A0000000000000000000E5550008E5550008CB
:1001B000E5550008E5550008E55500080000000079
:1001C00000000000E55500080000000000000000ED
:0801D000E5550008E5550008A3
:1001E00001F0FF01102A2BDB10F0070F08D010F8E8
:1001F000013B013A8B422DD010F0070F42B3F6D1EC
:10020000F0B441EA012141EA014122F007047FF004
:1002100000070023F0E80256083C85EA010586EA5B
:10022000010685FA47F5A3FA87F586FA47F6A5FA97
:1002300087F68EB9EED1F0BC01F0FF0102F00702A3
:1002400032B110F8013B013A83EA010313B1F8D14E
:100250000020704701387047002D06BF354603382F
:10026000073815F0010F07D1013015F4807F02BF68
:10027000013015F4C03F0130F0BC0138704700BFB9
:1002800053B94AB9002908BF00281CBF4FF0FF31FD
:100290004FF0FF3000F00CB8ADF1080C6DE904CE62
:1002A00005F05CFEDDF804E0DDE9022304B07047F0
:1002B000704700BF0348044B834202D0034B03B195
:1002C000184770475C0000205C0000200000000020
:1002D0000548064B1B1AD90F01EBA301491002D0A8
:1002E000034B03B1184770475C0000205C000020FE
:1002F0000000000010B5064C237843B9FFF7DAFF81
:10030000044B13B10448AFF300800123237010BDE8
:100310005C000020000000005462000808B5054B96
:100320001BB105490548AFF30080BDE80840FFF761
:10033000CFBF00BF00000000600000205462000832
:10034000F0B589B003AD0024039404940594069499
:100350000794214BDA6C42F02002DA64DA6C02F086
:1003600020020092009ADA6C42F00102DA64DA6C40
:1003700002F001020192019ADA6C42F00202DA64A0
:10038000DB6C03F002030293029B144E22465021C1
:10039000304601F064FD4FF480730393022304930D
:1003A00005940694079429464FF0904001F066FCAE
:1003B000082303930494012705972946304601F04A
:1003C0005DFC502303930497059406942946304618
:1003D00001F054FC09B0F0BD0010024000040048D8
:1003E00000B583B0164B9A6C42F004029A649A6C82
:1003F00002F004020092009A9A6C42F001029A64A0
:100400009B6C03F001030193019B002211460C2019
:1004100001F0EEFF0C2001F0FBFF002211460D2041
:1004200001F0E6FF0D2001F0F3FF002211460E203F
:1004300001F0DEFF0E2001F0EBFF03B05DF804FBDE
:100440000010024070470000014B01221A707047F3
:100450004F040020084B1B888B420BD006D9064B5B
:1004600000221A8002E00133034A1380024B1B88EA
:100470008B42F8D3704700BF78000020014B012267
:100480001A70704773050020014B01221A707047E3
:100490007305002072B6FEE700B58FB000230A9303
:1004A0000B930C930D930793089309930093019377
:1004B0000293039304930593069333484FF08042CD
:1004C00002604360836040F6FF72C2600361836133
:1004D00003F07EFC002846D14FF480530A930AA90A
:1004E000294803F0C5FD00283FD1274803F0A0FCB0
:1004F00000283CD1202307930023099307A9224811
:1005000003F00CFF002834D1602300934FF4FA73FA
:100510000193002202920423049369461A4803F0CF
:10052000FDFC40BB4FF47A730193042269461648E0
:1005300003F0F4FC08BB40F2DC5301930822694647
:10054000114803F0EBFCD0B94FF4FA6301930C228D
:1005500069460D4803F0E2FC98B90B4800F0D4FC62
:100560000FB05DF804FBFFF795FFFFF793FFFFF770
:1005700091FFFFF78FFFFFF78DFFFFF78BFFFFF76F
:1005800089FFFFF787FF00BF6802002008B5114808
:10059000114B0360114B4360002383600122C26052
:1005A000036143618361C361036203F03DF850B9A5
:1005B0000021084803F09CF838B90021054803F0F1
:1005C000C4F820B908BDFFF765FFFFF763FFFFF729
:1005D00061FF00BFB4020020005400409F6E9150A4
:1005E00000B589B000230493059306930793019304
:1005F000029303931348144A026044F29F1242602C
:1006000083606322C2600361836103F0E1FB90B900
:100610004FF48053049304A90A4803F029FD60B9FC
:1006200000230193039301A9064803F077FE30B934
:1006300009B05DF804FBFFF72DFFFFF72BFFFFF775
:1006400029FF00BF1C0200200004004010B592B03A
:1006500000240F9410941194089409940A940B9414
:100660000C940D940E9420222146684604F0F2FF6B
:100670002C484FF0A04303604FF440334360846044
:10068000C4600461446104238361047744770123D7
:10069000036280F824404FF4AC63C3624FF480637C
:1006A000036380F83840C46380F8404001F00EFFD7
:1006B00000282FD100230F930FA91A4802F028FF1A
:1006C00050BB194B08934FF440030993174B0A93FF
:1006D00001238DF82C304FF47D630C9330230D9360
:1006E00000230E9308A90F4802F0DCFBB0B90F4BB2
:1006F000009306230193052302937F23039304238E
:100700000493002305936946064802F09BF938B923
:1007100012B010BDFFF7BEFEFFF7BCFEFFF7BAFE3A
:10072000FFF7B8FED40300200000C07D0080F03E3B
:1007300000B589B020220021684604F08BFF2B48C9
:100740002B4B03604FF44033436000238360C3604E
:100750000361012242610822826103774377042208
:10076000026280F82430C362036380F83830C363C8
:1007700080F8403001F0AAFE00282DD11D4B0093D7
:100780000623019302937F230393042304930023FE
:1007900005936946154802F055F9F8B9164B0093D0
:1007A0000C2301936946114802F04CF9C0B9134B70
:1007B00000931223019369460C4802F043F988B96B
:1007C0000F4B0093182301936946084802F03AF949
:1007D00050B909B05DF804FBFFF75CFEFFF75AFE65
:1007E000FFF758FEFFF756FEFFF754FE68030020A0
:1007F000000100501000C0100800900C002090363E
:100800000000524708B51548154B03604FF41643D6
:10081000436000238360C36003610C2242618361F3
:10082000C36103624362836204F083FB70B90021F9
:100830000A4804F0F9FB58B90021084804F019FCF3
:1008400040B9064804F0D1FB30B908BDFFF722FEDD
:10085000FFF720FEFFF71EFEFFF71CFE3C01002005
:100860000038014010B59CB00024189419941A94D3
:100870001B941594169417940E940F94109411943D
:100880001294139414943422214601A804F0E2FE39
:100890003148324B036040F28F6343608460FF2332
:1008A000C36004614461846103F092FA002847D177
:1008B0004FF48053189318A9274803F0D9FB002858
:1008C00040D1254803F0B4FA00283DD10023159308
:1008D0001693179315A9204803F020FD002835D161
:1008E00060230E9300230F9310931193129313938D
:1008F000149308220EA9184803F010FB40BB0023F4
:10090000019302930393049305934FF400520692CC
:100910000793089309934FF000720A920B930C937C
:100920000D9301A90C4803F043FD98B90A480268E9
:10093000536C43F40043536400F0E6FA1CB010BD5E
:10094000FFF7A8FDFFF7A6FDFFF7A4FDFFF7A2FD47
:10095000FFF7A0FDFFF79EFDD0010020003401400D
:1009600010B594B006AC38220021204604F072FE87
:1009700000200190029003900490059001F056FC35
:10098000012306934FF48033079302230D93032230
:100990000E920F931C221092119304221292139321
:1009A000204600F0EFFBB0B90F230193032302931D
:1009B000002303930493059304210DEB010000F041
:1009C000C5FE50B900224FF080614FF4807000F0F6
:1009D0004BFE14B010BDFFF75DFDFFF75BFD00009F
:1009E00008B500F081FBFFF7BBFFFFF7A9FCFFF79D
:1009F000F7FCFFF751FDFFF7C9FDFFF7F1FDFFF72A
:100A000025FEFFF795FEFFF7FDFEFFF72BFF3F48A2
:100A100002F02CFC3E4C204603F038F83D4803F031
:100A200035F80021204603F0CFFB0421204603F0D7
:100A3000CBFB0821204603F0C7FB0C21204603F026
:100A4000C3FB354C204603F021F80821204603F073
:100A5000BBFB04220821206803F0A6FB04F06CFB1A
:100A600004F04AFC04F0D6FB04222C492C4802F086
:100A7000C5FC2C4B1978D9B12B4804F04DFB17E07D
:100A8000264C204604F070FB04222146244802F044
:100A9000B5FC264B00221A7012E004F035FC1BE076
:100AA000234A13780133DBB21370224B00221A70F1
:100AB000204B1B78002BFBD01C4B1B78002BDFD16D
:100AC0001D4B1888C0F3C70004F082FC04F074FBCF
:100AD0001A4B18780028E0D1154B1B780A2BDFD968
:100AE000134B00221A7004F0E1FC0821144801F0B5
:100AF000AFF910B9134B00221A700A4B197800296C
:100B0000D3D0094804F008FBCFE700BFD40300208E
:100B1000680200201C020020D001002050040020A8
:100B20006803002064040020680400204F040020B3
:100B30006805002069050020740500204D04002090
:100B4000000400484E040020FEE7FEE7FEE7FEE753
:100B5000FEE770477047704708B500F0D5FA08BD4A
:100B600008B5024801F000FB08BD00BF08030020E3
:100B700008B5024801F0F8FA08BD00BFDC0000200B
:100B800008B5024801F0F0FA08BD00BF7C00002063
:100B900008B5034801F0B6FD024801F0B3FD08BDF9
:100BA000D40300206803002008B50D4802F0B6FF0A
:100BB0000C4801F09DFD034680B20B4A12784AB101
:100BC0004FF0804300225A639A6304F007FC074BFE
:100BD000188008BD9BB24FF0804253639363F4E7E3
:100BE00068020020D40300204E0400207405002079
:100BF00008B5034802F092FF024B01221A7008BDAB
:100C00001C0200206905002008B5024803F02CFDF5
:100C100008BD00BF3C01002000B583B00B4B1A6E2D
:100C200042F001021A661A6E02F001020092009A66
:100C30009A6D42F080529A659B6D03F08053019348
:100C4000019B01F079FB03B05DF804FB001002404A
:100C500030B59BB00446002115911691179118915B
:100C60001991442204A804F0F5FC2368B3F1A04FC5
:100C700004D04B4A93423CD01BB030BD4FF40043EC
:100C800004934FF00053139304A800F085FE10BBAB
:100C9000444A136801331360012B1FD0424BDA6CB6
:100CA00042F00202DA64DB6C03F002030193019B61
:100CB00001231593032316930024179415A93B4889
:100CC00000F0DCFF22462146122001F091FB1220A9
:100CD00001F09EFBD0E7FFF7DDFBD9E7324BDA6C82
:100CE00042F40052DA64DB6C03F400530093009B7F
:100CF000D4E74FF4004304934FF00053139304A838
:100D000000F04AFE00283AD1264A136801331360E6
:100D1000012B37D0244BDA6C42F00102DA64DB6C31
:100D200003F001030393039BF0231593032316930E
:100D30000025179515A94FF0904000F09FFF1C4823
:100D40001C4B0360242343608560C56080230361DE
:100D50004FF4007343614FF400638361C561056222
:100D600001F0DCF8C8B9124B63659C6200221146A1
:100D7000122001F03DFB122001F04AFB7CE7FFF757
:100D800089FBC1E7084BDA6C42F40052DA64DB6C91
:100D900003F400530293029BBCE7FFF77BFBE2E7FF
:100DA00000010050400400200010024000040048F0
:100DB000080300201C0002402DE9F0419AB00446CF
:100DC000002115911691179118911991442204A8A8
:100DD00004F040FC2268254B9A4202D01AB0BDE8CC
:100DE000F0814023049304A800F0D6FD002839D1F7
:100DF0001F4CE36C43F00103E364E36C03F0010375
:100E00000193019BE36C43F00203E364E36C03F0A2
:100E100002030293029B4FF4004315934FF0120814
:100E2000CDF858800025179518950427199715AE09
:100E300031464FF0904000F021FF80231593CDF80C
:100E4000588017951895199731460A4800F016FFF3
:100E5000A36D43F40013A365A36D03F40013039380
:100E6000039BBBE7FFF716FBC2E700BF005400403F
:100E7000001002400004004800B585B00368B3F1DB
:100E8000804F08D01D4A934219D01D4A934229D061
:100E900005B05DF804FB03F504339A6D42F00102DE
:100EA0009A659B6D03F001030193019B002211469B
:100EB0001C2001F09DFA1C2001F0AAFAE8E7114B72
:100EC0009A6D42F002029A659B6D03F00203029351
:100ED000029B002211461D2001F08AFA1D2001F01C
:100EE00097FAD5E7074B1A6E42F400521A661B6E4A
:100EF00003F400530393039BCAE700BF00040040C0
:100F0000003401400010024000B589B00023039373
:100F100004930593069307930368B3F1804F05D0BC
:100F2000184A934219D009B05DF804FB03F5043365
:100F3000DA6C42F00102DA64DB6C03F00103019326
:100F4000019B0F230393022304930123079303A917
:100F50004FF0904000F092FEE5E70B4BDA6C42F068
:100F60000202DA64DB6C03F002030293029B20238B
:100F70000393022304930323079303A9034800F078
:100F80007DFED0E70034014000100240000400481C
:100F900030B599B004460021139114911591169122
:100FA0001791442202A804F055FB2268344B9A4260
:100FB00001D019B030BD0123029302A800F0ECFC6F
:100FC000002853D12F4B1A6E42F480421A661A6ED3
:100FD00002F480420092009ADA6C42F00102DA6474
:100FE000DB6C03F001030193019B4FF4C063139387
:100FF000022314930025159516930723179313A91D
:101000004FF0904000F03AFE1F48204B0360182339
:1010100043608560C5608023036145618561C5616A
:10102000056200F07BFF20BB174BC4F880309C6248
:101030001748184B03601923436010238360002373
:10104000C3608022026143618361C361036200F077
:1010500065FF88B90E4BE3679C620022114625208C
:1010600001F0C6F9252001F0D3F9A2E7FFF712FA43
:10107000A8E7FFF70FFAD7E7FFF70CFAEAE700BF98
:101080000038014000100240DC0000203000024027
:101090007C00002044000240104B1B680BB901206B
:1010A000704710B504464FF47A70B0FBF3F30C4A66
:1010B0001068B0FBF3F001F0AFF968B90F2C01D95B
:1010C00001200AE0002221464FF0FF3001F090F9A4
:1010D000044B1C60002000E0012010BD0000002037
:1010E000080000200400002010B5032001F06EF974
:1010F0000020FFF7D1FF10B10124204610BD0446A7
:10110000FFF78AFDF9E70000034A136803490968FD
:101110000B441360704700BF44040020000000200F
:10112000014B1868704700BF44040020124BDA6876
:1011300002F00302DB68C3F303130133032A11D067
:101140000E48B0FBF3F00C4BDB68C3F3062303FB44
:1011500000F0094BDB68C3F3416301335B00B0FB74
:10116000F3F070470648B0FBF3F0034BDB68C3F3C2
:10117000062303FB00F0ECE7001002400024F4001B
:1011800000366E01002800F04F8270B582B0044630
:10119000036813F0010F37D0A44A936803F00C03DF
:1011A000D26802F003020C2B23D0082B23D06368F3
:1011B000B3F5803F4ED0B3F5A02F51D09B4B1A68AA
:1011C00022F480321A601A6822F480221A6063685E
:1011D000002B52D0FFF7A4FF0546944B1B6813F475
:1011E000003F11D1FFF79CFF401B6428F5D9032075
:1011F00023E2032AD9D18D4B1B6813F4003F03D09F
:101200006368002B00F01282236813F0020F5DD098
:10121000864A936803F00C03D26802F003020C2B99
:101220003AD0042B3AD0E368002B75D07F4A13687C
:1012300043F480731360FFF773FF05467B4B1B6815
:1012400013F4806F5FD1FFF76BFF401B0228F5D9C5
:101250000320F2E1754A136843F480331360B6E764
:1012600003F18043A3F53C331A6842F480221A60EC
:101270001A6842F480321A60A9E7FFF751FF054669
:101280006A4B1B6813F4003FBED0FFF749FF401BB9
:101290006428F5D90320D0E1022AC2D1634B1B6830
:1012A00013F4806F03D0E368002B00F0C1815F4A24
:1012B000536823F0FE43216943EA016353605C4BAA
:1012C0001868FFF7E9FE002840F0B481236813F0A6
:1012D000080F4CD063699BB3544AD2F8943043F062
:1012E0000103C2F89430FFF71BFF05464F4BD3F8BC
:1012F000943013F0020F3AD1FFF712FF401B02287F
:10130000F4D9032099E1494A536823F0FE43216947
:1013100043EA01635360D9E7444A136823F48073B6
:101320001360FFF7FDFE0546404B1B6813F4806F0A
:10133000CCD0FFF7F5FE401B0228F5D903207CE155
:101340003A4AD2F8943023F00103C2F89430FFF700
:10135000E7FE0546354BD3F8943013F0020F06D064
:10136000FFF7DEFE401B0228F4D9032065E1236865
:1013700013F0040F00F081802C4B9B6D13F0805F05
:1013800036D12A4B9A6D42F080529A659B6D03F0DC
:1013900080530193019B0125264B1B6813F4807F2A
:1013A00028D0A368012B39D0052B45D01F4BD3F88B
:1013B000902022F00102C3F89020D3F8902022F070
:1013C0000402C3F89020A368002B43D0FFF7A8FEC7
:1013D0000646164BD3F8903013F0020F4CD1FFF7AE
:1013E0009FFE801B41F288339842F2D9032024E10A
:1013F0000025D1E70F4A136843F480731360FFF7A9
:101400008FFE06460B4B1B6813F4807FC9D1FFF794
:1014100087FE801B0228F5D903200EE1034AD2F88B
:10142000903043F00103C2F89030CCE70010024046
:101430000400002000700040884BD3F8902042F058
:101440000402C3F89020D3F8902042F00102C3F8C0
:101450009020B8E7FFF764FE0646804BD3F8903043
:1014600013F0020F08D0FFF75BFE801B41F28833B8
:101470009842F2D90320E0E0E5B9236813F0200F89
:1014800035D0A369E3B1754AD2F8983043F001032F
:10149000C2F89830FFF744FE0546704BD3F89830F9
:1014A00013F0020F23D1FFF73BFE401B0228F4D9B3
:1014B0000320C2E0694A936D23F080539365DCE713
:1014C000664AD2F8983023F00103C2F89830FFF74B
:1014D00027FE0546614BD3F8983013F0020F06D073
:1014E000FFF71EFE401B0228F4D90320A5E0E369A4
:1014F000002B00F0A180594A926802F00C020C2ADD
:1015000064D0022B13D0554A136823F08073136004
:10151000FFF706FE0446514B1B6813F0007F4ED0C8
:10152000FFF7FEFD001B0228F5D9032085E04B4A9A
:10153000136823F080731360FFF7F2FD0546474BF5
:101540001B6813F0007F06D0FFF7EAFD401B02285E
:10155000F5D9032071E0414AD36841491940236A13
:10156000606A013843EA0013A06A43EA0023206B53
:101570004008013843EA4053606B4008013843EAB1
:101580004063E06A43EAC0631943D160136843F0E3
:1015900080731360D36843F08073D360FFF7C0FD9E
:1015A00004462E4B1B6813F0007F06D1FFF7B8FDF1
:1015B000001B0228F5D903203FE000203DE0274A28
:1015C000D168284B0B40D360002036E0012B36D089
:1015D000224BDB6803F00301226A914231D103F010
:1015E000F002616A0139B2EB011F2CD103F4FE4213
:1015F000A16AB2EB012F28D103F07842E16AB2EB85
:10160000C16F24D103F4C001226B5208013AB1EB3F
:10161000425F1ED103F0C063626B5208013AB3EB24
:10162000426F18D1002008E001207047012004E03B
:10163000012002E0012000E0002002B070BD012086
:10164000FBE70120F9E70120F7E70120F5E701209A
:10165000F3E70120F1E70120EFE700BF00100240AF
:101660000C809F01FCFFEEFE70B586B00C4615465F
:1016700002230293032304930023039300F0805674
:10168000C0F3034C0CF5901E0D4AD36C012101FAF6
:101690000CF10B43D36483B20193C0F30750059060
:1016A00001A94FEA8E2000F0E9FA36B9044A93689E
:1016B00023F0FE432C431C43946006B070BD00BF72
:1016C000001002401E4B9B6803F00C03042B33D028
:1016D0001B4B9B6803F00C03082B2FD0184B9B6807
:1016E00003F00C030C2B01D000207047144BDA6878
:1016F00002F00302DB68C3F303130133032A11D0A2
:101700001048B0FBF3F00E4BDB68C3F3062303FB7A
:1017100000F00B4BDB68C3F3416301335B00B0FBAC
:10172000F3F070470848B0FBF3F0054BDB68C3F3F8
:10173000062303FB00F0ECE70248704702487047BD
:10174000001002400024F40000366E01002800F072
:10175000E680F8B50C460546744B1B6803F00F0392
:101760008B420BD2714A136823F00F030B431360B3
:10177000136803F00F038B4240F0D3802E6816F0FD
:1017800001065FD06B68032B2FD0022B4DD0684B26
:101790001B6813F4806F00F0C680FFF793FF654B62
:1017A00098424DD9624A936823F0F00343F08003D6
:1017B000936080265E4A936823F0030369680B43B5
:1017C0009360FFF7ADFC0746594B9B6803F00C0391
:1017D0006A68B3EB820F35D0FFF7A2FCC01B41F261
:1017E00088339842F0D9032078E0514B1B6813F0FE
:1017F000007F01D1012071E0FFF798FC4D4B98422A
:101800001AD94B4B9B6813F0F00F05D02E6816F0D9
:101810000206CFD0AB688BB9454A936823F0F0033A
:1018200043F0800393608026C4E7414B1B6813F4A8
:10183000003FB2D1012051E00026BBE70026B9E706
:101840000026B7E72B6813F0020F48D013F0040FFF
:1018500004D0374A936843F4E06393602B6813F035
:10186000080F06D0324A936823F47C5343F4E063B4
:1018700093602F4A936823F0F003A9680B439360A9
:101880002A4B1B6803F00F03A34230D82B6813F0D8
:10189000040F06D0264A936823F4E063E9680B43FB
:1018A00093602B6813F0080F07D0214A936823F444
:1018B0006053296943EAC1039360FFF703FF1C4BA0
:1018C0009B68C3F303131C4AD35C03F01F03D84087
:1018D0001A4B18601A4B1868FFF7DEFBF8BD802E14
:1018E000CED1134A936823F0F0039360C8E70F4A00
:1018F000136823F00F0323431360FFF711FC064620
:101900000A4B1B6803F00F03A342BFD0FFF708FC8C
:10191000801B41F288339842F2D90320DEE7012090
:1019200070470120DAE70120D8E700BF002002401D
:101930000010024000B4C4049C62000808000020AB
:1019400004000020014B1868704700BF0800002009
:1019500008B5FFF7F7FF054B9B68C3F30223044A62
:10196000D35C03F01F03D84008BD00BF0010024045
:101970009462000808B5FFF7E5FF054B9B68C3F3C9
:10198000C223044AD35C03F01F03D84008BD00BF44
:101990000010024094620008F0B583B0044603686A
:1019A00013F4002F69D0AE4B9B6D13F0805F1ED1F6
:1019B000AB4B9A6D42F080529A659B6D03F0805359
:1019C0000193019B0126A74A136843F480731360B7
:1019D000FFF7A6FB0546A34B1B6813F4807F08D1D5
:1019E000FFF79EFB401B0228F5D9032502E00026E5
:1019F000E9E7002545BB9A4BD3F8903013F44073C8
:101A000018D0226C9A4212D0954AD2F8903023F422
:101A10004073D2F8901041F48031C2F89010D2F89F
:101A2000901021F48031C2F89010C2F8903013F079
:101A3000010F10D145B98A4AD2F8903023F440738F
:101A4000216C0B43C2F89030C6B1854A936D23F0E8
:101A50008053936512E0FFF763FB0746804BD3F892
:101A6000903013F0020FE5D1FFF75AFBC01B41F293
:101A700088339842F2D90325DCE70025236813F068
:101A8000010F08D0764AD2F8883023F0030361684A
:101A90000B43C2F88830236813F0020F08D0704A55
:101AA000D2F8883023F00C03A1680B43C2F88830C9
:101AB000236813F0040F08D0694AD2F8883023F065
:101AC0003003E1680B43C2F88830236813F0080F35
:101AD00008D0634AD2F8883023F0C00321690B4351
:101AE000C2F88830236813F0200F08D05C4AD2F87F
:101AF000883023F4406361690B43C2F8883023685F
:101B000013F0400F08D0564AD2F8883023F44053DF
:101B1000A1690B43C2F88830236813F0800F08D006
:101B20004F4AD2F8883023F44043E1690B43C2F8AE
:101B30008830236813F4807F08D0494AD2F888306F
:101B400023F44033216A0B43C2F88830236813F42E
:101B5000007F08D0424AD2F8883023F44023616ADB
:101B60000B43C2F88830236813F4806F0CD03C4AD2
:101B7000D2F8883023F44013A16A0B43C2F88830AE
:101B8000A36AB3F5801F57D0236813F4006F0CD0FD
:101B9000334AD2F8883023F44003E16A0B43C2F899
:101BA0008830E36AB3F5800F4BD0236813F4805F6D
:101BB0000CD02B4AD2F8883023F04073216B0B43B2
:101BC000C2F88830236BB3F1807F3FD0236813F4D1
:101BD000005F0CD0224AD2F8883023F04063616B5A
:101BE0000B43C2F88830636BB3F1006F33D02368C6
:101BF00013F4804F0CD01A4AD2F8883023F0406397
:101C0000A16B0B43C2F88830A36BB3F1006F2BD0EC
:101C1000236813F4004F0CD0114AD2F8883023F017
:101C20004053E16B0B43C2F88830E36BB3F1805F44
:101C30001FD0284603B0F0BDD36843F48013D360AF
:101C4000A2E7D36843F48013D360AEE7D36843F4CC
:101C50008013D360BAE7D36843F48013D360C6E738
:101C60000010024000700040D36843F48013D3603A
:101C7000CEE7D36843F48033D360DAE7F0B583B0BE
:101C8000002362E085685E000324B44025EA040571
:101C9000CC68B4402C438460456825EA0C054C6848
:101CA000C4F300149C402C4344605FE0DD08083519
:101CB00050F8254003F0070C4FEA8C0C4FF00F0E44
:101CC0000EFA0CFE24EA0E0E0C6904FA0CF444EA37
:101CD0000E0440F8254060E0052400E0002404FAEA
:101CE0000EF42C430CF1020C554D45F82C40554C8C
:101CF000A568D44325EA02064F6817F4801F01D077
:101D000042EA05064F4DAE60ED6804EA05064F68ED
:101D100017F4001F01D042EA05064A4DEE606D68D7
:101D200004EA05064F6817F4003F01D042EA0506B1
:101D3000444D6E602D682C404E6816F4803F01D0F3
:101D400042EA05043F4A146001330A6832FA03F498
:101D500074D04FF0010C0CFA03FC1CEA0202F3D021
:101D60004C6804F00304013C012C8BD94C6804F04E
:101D70000304032C0CD0C4685D004FF0030C0CFA74
:101D800005FC24EA0C0C8C68AC4044EA0C04C460EA
:101D90004C6804F00304022C88D004684FEA430E18
:101DA0004FF0030C0CFA0EFC24EA0C0C4C6804F007
:101DB000030404FA0EF444EA0C0404604C6814F4BE
:101DC000403FC1D0204C256E45F001052566246EAC
:101DD00004F001040194019C4FEA930C0CF10205FC
:101DE000174C54F8255003F0030E4FEA8E0E0F24C3
:101DF00004FA0EF425EA0405B0F1904F3FF46EAFFB
:101E0000124CA04212D004F58064A04210D004F518
:101E10008064A0420ED004F58064A0420CD004F58A
:101E20008064A0423FF458AF062458E7012456E7E7
:101E3000022454E7032452E7042450E703B0F0BD22
:101E4000000001400004014000100240000400486E
:101E50000369194201D001207047002070470AB180
:101E6000816170478162704730B4C46C056D6560F4
:101E7000446D14B1846DC56D6560446C04F01F0C35
:101E8000012404FA0CF4056C6C60046863608368D8
:101E9000102B05D0036899600368DA6030BC704786
:101EA00003689A600368D960F8E7000003680C4A89
:101EB000934213D80B49DBB2083B0B4AA2FB032326
:101EC000426C22F003020A448264084AC264C3F3EB
:101ED0000413012202FA03F3036570470449EAE799
:101EE0000704024000080240CDCCCCCC8008024060
:101EF000200802400379074A1A4492004265064AC4
:101F00008265013B03F01F03012202FA03F3C3655C
:101F1000704700BF3F82001040090240002859D09E
:101F200010B5044602682C4B9A423BD82B4B134405
:101F30002B49A1FB03131B099B004364294B03643A
:101F4000022384F8253011686FF30E11A368E0684E
:101F500003432069034360690343A0690343E069C5
:101F60000343206A03430B4313602046FFF79EFFA1
:101F7000A368B3F5804F20D0A36C22791A60E36C7C
:101F8000226D5A606368013B032B19D900236365F6
:101F9000A365E3650020E063012384F8253084F81D
:101FA000240010BD104B13440D49A1FB03131B0962
:101FB0009B0043640D4B0364C2E700236360DBE7CF
:101FC0002046FFF797FF636D00221A60A36DE26D54
:101FD0005A60DFE70120704707040240F8FFFDBFA9
:101FE000CDCCCCCC00000240F8FBFDBF0004024089
:101FF00038B5044690F82400012840D0012084F828
:10200000240094F82500012804D0002384F824300B
:10201000022038BD022084F825000020E0632568F6
:10202000286820F0010028602046FFF71DFF236B81
:10203000D3B12268136843F00E031360A36C1A68CF
:1020400012F4803F03D01A6842F480721A60636D04
:102050001BB11A6842F480721A602268136843F058
:10206000010313600020D4E72268136823F00403FF
:1020700013602268136843F00A031360DEE702204E
:10208000C7E7034690F82520022A09D00422C2633C
:102090000120012283F82520002283F824207047A4
:1020A00001680A6822F00E020A60816C0A6822F454
:1020B00080720A6001680A6822F001020A60426CBC
:1020C00002F01F01006C01228A404260DA6C196D37
:1020D00051605A6D42B1116821F4807111609A6D9E
:1020E000D96D51600020D4E70020D2E708B590F800
:1020F0002530022B09D00423C363012380F8253047
:10210000002280F82420184608BD0268136823F0D6
:102110000E0313600268136823F001031360826CDE
:10212000136823F480731360436C03F01F02016C87
:10213000012393404B60C36C026D5A60436D33B111
:102140001A6822F480721A60836DC26D5A6001238E
:1021500080F82530002380F82430836B13B1984732
:102160000020D1E70020CFE738B5036C1968046878
:102170002568436C03F01F0304229A400A4215D0DD
:1021800015F0040F12D0236813F0200F03D1236839
:1021900023F004032360436C03F01F02016C04234B
:1021A00093404B60036B03B1984738BD02229A40BD
:1021B0000A421CD015F0020F19D0236813F0200F2B
:1021C00006D1236823F00A032360012380F8253019
:1021D000436C03F01F02016C022393404B60002309
:1021E00080F82430C36A002BDFD09847DDE708224F
:1021F00002FA03F30B42D8D015F0080FD5D02368AC
:1022000023F00E032360436C03F01F03016C0122D3
:1022100002FA03F34B60C26380F82520002380F8A4
:102220002430436B002BC0D09847BEE7002836D13E
:102230003E4B1B6803F4C063B3F5806F08D03B4A84
:10224000D2F8803023F48073C2F8803000207047C9
:10225000364AD2F8803023F48073C2F88030136895
:1022600023F4C06343F400731360314B1B683222C4
:1022700002FB03F32F4AA2FB03239B0C013300E074
:10228000013B2A4A526912F4806F01D0002BF7D12A
:10229000264B5B6913F4806F44D100207047B0F582
:1022A000007F08D0214A136823F4C06343F480639D
:1022B0001360002070471D4B1B6803F4C063B3F527
:1022C000806F08D0194AD2F8803043F48073C2F886
:1022D000803000207047154AD2F8803043F4807374
:1022E000C2F88030136823F4C06343F400731360B2
:1022F0000F4B1B68322202FB03F30E4AA2FB03239F
:102300009B0C013300E0013B084A526912F4806FD4
:1023100001D0002BF7D1054B5B6913F4806F03D11B
:102320000020704703207047032070470070004072
:102330000800002083DE1B43024A936843F4804375
:102340009360704700700040002807DB00F01F0218
:10235000400901239340024A42F82030704700BFF1
:1023600000E100E0002808DB0901C9B200F160408B
:1023700000F5614080F80013704700F00F0009017C
:10238000C9B2014B1954704714ED00E000B500F0DC
:102390000700C0F1070CBCF1040F28BF4FF0040C7C
:1023A000031D062B0FD9C31E4FF0FF3E0EFA0CF093
:1023B00021EA000199400EFA03FE22EA0E0241EAE8
:1023C00002005DF804FB0023EEE70000074AD36833
:1023D00023F4E0631B041B0C000200F4E0600343E1
:1023E00043F0BF6343F40033D360704700ED00E077
:1023F00010B50446054BD868C0F30220FFF7C6FFAE
:1024000001462046FFF7AEFF10BD00BF00ED00E023
:1024100008B5FFF799FF08BD0138B0F1807F0BD2F6
:102420004FF0E0235861054AF02182F82310002084
:10243000986107221A6170470120704700ED00E0A3
:1024400010B430300B0A9B0003F00C03C45801F0A9
:102450001F014FF01F0C0CFA01FC24EA0C0CC2F314
:1024600084628A404CEA0202C2505DF8044B704715
:1024700010B414304B0E9B0003F00403C458C1F396
:1024800004514FF0070C0CFA01FC24EA0C0C8A40B2
:102490004CEA0202C2505DF8044B704700B50C30A4
:1024A000C1F3015C41F3000303F024039C4450F8A2
:1024B0002C3021F0024E2EF4601E23EA0E03114050
:1024C0000B4340F82C305DF804FB000030B583B0BE
:1024D00000230193002800F0FF800446C36D13B36E
:1024E00023689A6812F0005F05D09A6822F02042B3
:1024F00022F03F029A602268936813F0805F1FD138
:10250000936823F0104323F03F0343F0805393601C
:10251000724B1B689B09724AA2FB03239B09013380
:102520005B00019309E0FEF793FB0023236684F828
:102530005830D5E7019B013B0193019B002BF9D15A
:102540002268936813F0805F40F09280E36D43F05F
:102550001003E365236E43F00103236601209368B3
:1025600013F0040300D00123E16D11F0100F40F0CF
:10257000AC80002B40F0A980E36D23F4817343F01D
:102580000203E365936813F0010F13D14FF0A043EA
:102590009B6813F0010300D00123524A926812F0A5
:1025A000010F07D133B963684F498A6822F47C125E
:1025B00013438B60627FE36B43EA4233E268134369
:1025C000A268134394F8242043EA0243012A51D01D
:1025D000E26A22B102F47872216B0A431343216844
:1025E000CD68424A2A401A43CA602268136923F020
:1025F0004063616B0B4313612268936813F0080317
:1026000000D001232BBB237F94F83810490041EA06
:102610008331D36823F4804323F002030B43D36058
:10262000236963B32268136943F48033136122681A
:10263000D2F8C0306FF30D0321690B43C2F8C030EC
:1026400094F84030012B27D02268136923F001034E
:1026500013616369012B2FD02268136B23F00F03E2
:102660001363E36D23F0030343F00103E36531E0FB
:10267000002074E7A26A013A43EA4243A8E72268CD
:10268000136923F4803313612268D2F8C0306FF3EA
:102690000D03C2F8C030D3E721680B696FF38A03DA
:1026A000626CA56C2A43E56C2A43256D2A431343CB
:1026B00043F001030B61CCE721680B6B23F00F03A0
:1026C000226A013A13430B63CBE7E36D43F0100337
:1026D000E365012003B030BD0120FBE708000020C6
:1026E000632D3E0500010050000300500740F0FF3D
:1026F0000368186C7047704708B5806AFFF7FBFFE6
:1027000008BD7047F8B5044603681F685D689A4BBA
:102710009E6806F01F0617F0020F10D015F0020F8A
:102720000DD0C36D13F0100F03D1C36D43F40063DC
:10273000C365204600F0EAFE236802221A6017F003
:10274000040F02D015F0040F05D117F0080F4DD07B
:1027500015F0080F4AD0E36D13F0100F03D1E36DAD
:1027600043F40073E3652368DA6812F4406F37D1ED
:10277000824A934227D01A46934207D0092E25D881
:1027800040F22121F14011F0010F1FD0DA6812F45C
:10279000005F25D11A6812F0080F21D09A6812F054
:1027A000040F15D15A6822F00C025A60E36D23F42D
:1027B0008073E365E36D13F4805F11D1E36D43F043
:1027C0000103E3650CE04FF0A042D5E7D268DEE7F5
:1027D000E36D43F01003E365236E43F001032366CA
:1027E0002046FDF731FE23680C221A6017F0200FF7
:1027F00002D015F0200F05D117F0400F5CD015F076
:10280000400F59D0E36D13F0100F03D1E36D43F483
:102810000053E3652368DA6C12F4C07F12D1012102
:10282000DA6812F4406F0FD10120544A93420DD060
:102830001A4693420DD066B1062E0AD0072E08D054
:10284000D26807E00021EBE70020EEE74FF0A0425E
:10285000EFE7DA6851B312F0007F03D030B312F41F
:10286000005F23D1196811F0400F1FD012F4001F30
:102870001CD19A6812F0080F10D15A6822F0600239
:102880005A60E36D23F48053E365E36D13F4807FB6
:102890000CD1E36D43F00103E36507E0E36D43F022
:1028A0001003E365236E43F001032366204600F026
:1028B00029FE236860221A6017F0800F02D015F0FD
:1028C000800F2FD117F4807F02D015F4807F34D190
:1028D00017F4007F02D015F4007F3AD117F0100FE3
:1028E00019D015F0100F16D0E36B33B1002E3CD089
:1028F000214B9B6813F4604F0AD0E36D43F480636F
:10290000E365236E43F0020323662046FFF7F9FEDA
:10291000236810221A6017F4806F02D015F4806FBC
:102920002ED1F8BDE36D43F48033E3652046FDF717
:1029300089FD236880221A60C4E7E36D43F4003305
:10294000E365204600F0E0FD23684FF480721A60D2
:10295000BEE7E36D43F48023E365204600F0D5FD38
:1029600023684FF400721A60B8E72368DB6813F03D
:10297000010FCDD0C1E700BF00030050000100509F
:10298000E36D43F48043E365236E43F0080323665D
:1029900023684FF480621A60204600F0B4FDC0E75F
:1029A00008B50346806AC26D12F0500F30D1C36D76
:1029B00043F40073C36503681A6812F0080F14D05B
:1029C000DA6812F4406F20D1DB6813F4005F1CD189
:1029D000C36D23F48073C365C36D13F4805F14D19A
:1029E000C36D43F00103C3650FE0DB6813F0020F12
:1029F0000BD1C36D23F48073C365C36D13F4805F83
:102A000003D1C36D43F00103C365FDF71DFD08BD90
:102A1000C26D12F0100F04D1426D526B18469047F0
:102A2000F5E7FFF76EFEF2E708B5806AC36D43F085
:102A30004003C365036E43F004030366FFF761FEC2
:102A400008BD0000F0B583B00023019390F8583022
:102A5000012B00F01C8204460D46012380F85830FB
:102A60000068836813F0040F09D0E36D43F020037E
:102A7000E3650120002384F8583003B0F0BD0A68F4
:102A80004968FFF7DDFC2068836813F0040300D079
:102A90000123866816F0080600D00126002B3ED1DF
:102AA000002E3CD1AA68B2F1004F6FD02968FFF721
:102AB000DFFC2268536923F000435361696922688F
:102AC000D368C3F3C1035B009940286904286AD026
:102AD000603252F82070AB4B3B402F6807F0F84C47
:102AE00041EA0C010B4343F0004342F820302368D5
:102AF0002869AA69603353F8201021F080710A43D5
:102B000043F82020236829692A7F012A48D06033AE
:102B100053F8212022F00072324343F8212022682A
:102B2000936813F0010F16D12B68E868D2F8B01043
:102B3000C3F3120621EA060100F018069248F0409D
:102B40000340C3F312030B43C2F8B030EA688F4B63
:102B50009A4200F08F802B688D4A134200F08F81DB
:102B60008C4A926802F0E0718B48834200F03E810B
:102B70008A48834200F03A818948834200F05C81B0
:102B80008848834200F06A81002073E700222968A8
:102B9000FFF76EFC2268536943F0004353618DE7F1
:102BA0004FF00076B3E7136E116EC1F384612B68AA
:102BB000C3F3120078BBC3F38463994233D0216816
:102BC0004B6E4A6EC2F384622B68C3F3120078BB6B
:102BD000C3F384639A4233D021688B6E8A6EC2F34A
:102BE00084622B68C3F3120078BBC3F384639A42F8
:102BF00033D02168CB6ECA6EC2F384622B68C3F3F4
:102C0000120078BBC3F384639A4288D1CB6E23F061
:102C10000043CB6683E793FAA3F313B1B3FA83F3CC
:102C2000CBE72023C9E7136E23F000431366C6E702
:102C300093FAA3F313B1B3FA83F3CBE72023C9E7E5
:102C40004B6E23F000434B66C6E793FAA3F313B130
:102C5000B3FA83F3CBE72023C9E78B6E23F000435D
:102C60008B66C6E793FAA3F313B1B3FA83F3CBE70A
:102C70002023C9E720682B68C3F3120626BB9A0EEF
:102C8000013202F01F02092A8CBF00220122002A11
:102C900052D046BB990E0131890601F0F84176BB4E
:102CA0009F0E013707F01F070122BA401143AEBB48
:102CB0009B0E013303F01F0303EB43031B05194372
:102CC000AA68FFF7D5FB46E793FAA3F24AB1B2FA36
:102CD00082F2013202F01F02092A8CBF0022012277
:102CE000D5E72022F5E793FAA3F131B1B1FA81F1EA
:102CF0000131890601F0F841D1E72021F8E793FA84
:102D0000A3F24AB1B2FA82F2013202F01F024FF08E
:102D1000010C0CFA02F2C9E72022F5E793FAA3F3BB
:102D200043B1B3FA83F3013303F01F0303EB43030F
:102D30001B05C4E72023F6E7CEB9990E01318906B9
:102D400001F0F84196BB9F0E013707F01F070122E3
:102D5000BA401143CEBB9B0E013303F01F0303EBBC
:102D600043031E3B1B0543F000731943A8E793FA86
:102D7000A3F1C9B1B1FA81F10131890601F0F8413D
:102D8000E0E700BF00F0FF03FFFF070000007F4007
:102D90000000088000030050000021C31000C09014
:102DA000000052C7000084CB2021E5E793FAA3F28C
:102DB0004AB1B2FA82F2013202F01F024FF0010C66
:102DC0000CFA02F2C5E72022F5E793FAA3F35BB110
:102DD000B3FA83F3013303F01F0303EB43031E3BFA
:102DE0001B0543F00073C0E72023F3E712F4000F44
:102DF0007FF4C2AE2368B3F1A04F01D0002039E6C2
:102E000041F40001234A936823F0E0731943916071
:102E1000214B1B689B09214AA2FB03239B09013319
:102E200003EB43039B000193019B1BB1019B013BFF
:102E30000193F9E700201DE612F0807F7FF4A0AE39
:102E40002268174B9A421CD041F08071114A936856
:102E500023F0E0731943916000200BE612F4800F19
:102E600011D122680E4B9A420FD041F480030949D8
:102E70008A6822F0E07213438B600020FAE500209C
:102E8000F8E50020F6E50020F4E50020F2E5022058
:102E9000F3E500BF0003005008000020632D3E054D
:102EA0000001005038B590F85830012B00F06781D0
:102EB00004460D46012380F858300068836813F0FB
:102EC000040300D00123826812F0080200D001221E
:102ED0007BBB72BB2968AB4B994262D06B68B3F184
:102EE000A07F00F0E28000F2D580B3F5400F00F043
:102EF000DC80B3F1807F03D0B3F5000F40F0D180C8
:102F0000A14AFFF7CBFA2A68A04B9A4200F004814D
:102F1000E36D23F48023E36523684FF400721A60A5
:102F20002B7B012B00F00F812268536823F4007380
:102F300053602B68934A934200F00B812068C2686B
:102F400002F01802182A00F013812969C268C2F33E
:102F5000C102C2F10202520002F01E0221FA02FC7A
:102F6000C26802F01802182A00F006816969C26876
:102F7000C2F3C102C2F10202520002F01E02D140AD
:102F8000206820301B0D9B0003F00C03C25802F098
:102F9000F02241EA0C410A43C250002084F8580054
:102FA00038BD6B68B3F1A07F48D011D8B3F5400F9E
:102FB00021D0B3F1807F4ED0B3F5000F5DD1C3684F
:102FC00023F0FB4323F4800343F40003C3601EE0BB
:102FD000B3F1C07F48D0B3F1E07F4ED1AA68C36897
:102FE00023F0FB4323F4800302F0F84242F0E07246
:102FF0001343C3600BE0AA68C36823F0FB4323F4C8
:10300000800302F0F84242F440021343C360226896
:10301000136A23F4E043A9690B431362E36D23F4BD
:103020008033E365236880221A602B7B012B2BD031
:103030002268536823F0800353607AE7AA68C36864
:1030400023F0FB4323F4800302F0F84242F0A07225
:103050001343C360DBE7C36823F0FB4323F480031F
:1030600043F08073C360D2E7C36823F0FB4323F4CB
:10307000800343F0C073C360C9E7C36823F0FB4318
:1030800023F48003C360C2E72268536843F08003DF
:1030900053604EE7B3F1C07F3FF432AFB3F1E07F4E
:1030A00003D00022FFF7FAF92DE7384B99420DD0F3
:1030B000AB68C3F312021ABBC3F3846301229A40C4
:1030C000D0F8A4301343C0F8A4301CE7AB68C3F3B6
:1030D00012024AB9C3F3846301229A40D0F8A030A7
:1030E0001343C0F8A0300EE793FAA3F333B1B3FA59
:1030F00083F303F01F0301229A40EFE72023F8E750
:1031000093FAA3F333B1B3FA83F303F01F0301225D
:103110009A40D5E72023F8E7E36D23F40033E36515
:1031200023684FF480721A602B7B012B05D0226834
:10313000536823F480735360FBE62268536843F4BA
:1031400080735360F5E62268536843F4007353605C
:10315000EFE629692068C268C2F3C102520001FA91
:1031600002FC6969C268C2F3C1025200914007E7DC
:103170002A694FEA820CF3E66969890000E70220B8
:103180000EE700BF0000C07DFFFF8701FFFF1700B3
:1031900030B583B00023019303689A6812F0010FE1
:1031A00058D1044699682D4A114219D19A6822F0E3
:1031B000004222F03F0242F001029A60284B9B68D5
:1031C00013F4000F1CD0274B1B689B09264AA2FB57
:1031D00003239B09013303EB43039B0001930CE0A2
:1031E000C36D43F01003C365036E43F00103036630
:1031F000012030E0019B013B0193019B002BF9D1A1
:10320000FDF78EFF054623681A6812F0010F1FD1E3
:103210009A6812F0010F07D19A6822F0004222F05A
:103220003F0242F001029A60FDF77AFF431B022B36
:10323000E9D923681B6813F0010FE4D1E36D43F073
:103240001003E365236E43F001032366012002E0CF
:10325000002000E0002003B030BD00BF3F00008030
:103260000003005008000020632D3E0538B5614B77
:103270009D6803689B6813F0040F40F0B680044615
:1032800005F01F0590F85830012B00F0B0800123A5
:1032900080F85830FFF77CFF002840F0A280E36DF3
:1032A00023F4706323F0010343F48073E365236820
:1032B000514A934257D01A46934200D01DB9E26D4D
:1032C00022F48012E265E26D12F4805F4ED0226E2D
:1032D00022F0060222661C221A60002384F858306D
:1032E0002268536823F01C035360A369082B40D065
:1032F0002268536843F004035360E36B23B92268E8
:10330000536843F01003536023683B4A934236D01E
:103310001A46934207D0092D3ED840F22121E940B8
:1033200011F0010F38D0DA6812F0007F11D0E26D91
:1033300022F4405242F48052E265A269082A21D068
:103340005A6822F040025A602268536843F0200312
:1033500053602268936823F0004323F03F0343F057
:103360000403936042E04FF0A042A5E700222266EA
:10337000B1E72268536843F008035360BDE74FF09C
:10338000A042C6E75A6822F020025A6022685368B9
:1033900043F040035360DCE7E16D41F48011E165E7
:1033A000D26812F0007F21D0E26D22F4405242F444
:1033B0008052E265A269082A09D05A6822F04002C8
:1033C0005A602268536843F0200353600EE05A6845
:1033D00022F020025A602268536843F04003536091
:1033E00004E0002384F8583000E0022038BD0220B9
:1033F000FCE700BF0003005000010050F8B5044690
:103400003B4B9D680068806810F0040F6CD10E463D
:10341000174605F01F0594F85830012B66D001239C
:1034200084F85830092D05D840F22123EB4013F0E1
:10343000010F04D1002384F85830012055E02046C4
:10344000FFF7A6FE00284BD1E36D23F4706323F051
:10345000010343F48073E3652368264A934239D01D
:103460001A46934200D01DB9E36D23F48013E3653F
:10347000E36D13F4805F30D0236E23F006032366E0
:10348000636D1D4ADA62636D1C4A1A63636D1C4AE0
:103490005A6323681C221A60002384F8583022687B
:1034A000536843F0100353602268D36843F001036C
:1034B000D36021683B4632464031606DFEF798FD8F
:1034C0002268936823F0004323F03F0343F0040392
:1034D00093600AE04FF0A042C3E700232366CFE7E2
:1034E000002384F8583000E00220F8BD0220FCE7F9
:1034F0000003005000010050A1290008F92600082F
:10350000292A0008704770477047704770470000CD
:1035100090F85820012A00F0818010B49DB0034635
:10352000012280F858200022189219920068B0F108
:10353000A04F38D000220192019A002A36D092681A
:1035400012F0040200D00122806810F0040F51D163
:10355000002A4FD10A68002A31D0314CA26822F4E7
:103560006042486893F838C040EA4C300243A26099
:103570004FF0A042926812F0010200D001222948C7
:10358000806810F0010F41D1002A41D1244CA2687B
:1035900022F4716222F00F020868896801430A432D
:1035A000A26000202BE01F4A0192C5E7DA6D42F0CD
:1035B0002002DA65002283F85820012022E0184911
:1035C0008A6822F460428A604FF0A042926812F04A
:1035D000010200D001221349896811F0010F19D1AD
:1035E000D2B90F498A6822F4716222F00F028A6010
:1035F000002004E0DA6D42F02002DA6501200022AA
:1036000083F858201DB05DF8044B70470020F6E7A2
:103610000020F4E70020F2E70020F0E702207047E6
:10362000000300500001005000285FD010B5044690
:1036300090F84130002B48D0242384F84130226890
:10364000136823F0010313606368226823F070633A
:1036500013612268936823F400439360E368012BAD
:1036600038D0A368226843F404439360E368022BD4
:1036700036D02268536823F400635360226853688D
:1036800043F0007343F4004353602268D36823F48B
:103690000043D360236962691343A169226843EA46
:1036A0000123D360E369216A22680B431360226817
:1036B000136843F00103136000206064202384F842
:1036C0004130206384F8420010BD80F84030FDF79F
:1036D00073FBB1E7A368226843F400439360C5E736
:1036E0002268536843F400635360C7E701207047C2
:1036F000034690F84120202A23D190F84020012A47
:1037000021D0012280F84020242280F84120006846
:10371000026822F0010202601868026822F48052F6
:103720000260186802680A43026019680A6842F079
:1037300001020A60202283F84120002083F8400023
:1037400070470220704702207047034690F84120DE
:10375000202A21D190F84020012A1FD0012280F890
:103760004020242280F841200068026822F00102F3
:1037700002601868026822F4706242EA0122026064
:1037800019680A6842F001020A60202283F8412089
:10379000002083F8400070470220704702207047E5
:1037A00030B4026A036A23F0010303624468836948
:1037B00023F4803323F073030D681D4322F00202CB
:1037C0008B6813431C4A90420FD002F5006290426E
:1037D0000BD002F54062904207D002F58062904221
:1037E00003D002F58062904205D123F00803CA6835
:1037F0001A4322F00403104A90420FD002F50062EF
:1038000090420BD002F54062904207D002F58062F0
:10381000904203D002F58062904205D124F44074B6
:103820004A6922438C691443446085614A68426353
:10383000036230BC704700BF002C014030B4036A03
:10384000026A22F4807202624468C26922F4803201
:1038500022F073020D68154323F400738A6843EA6B
:103860000223184A904203D002F50062904206D12A
:1038700023F40063CA6843EA022323F48063114AF5
:1038800090420FD002F5006290420BD002F54062E8
:10389000904207D002F58062904203D002F5806228
:1038A000904207D124F440524C6942EA04128C69D8
:1038B00042EA04144460C5614A68C263036230BCD2
:1038C000704700BF002C014030B4036A026A22F442
:1038D000805202624468C26922F0807222F4E64299
:1038E0000D6842EA052223F400538D6843EA05334C
:1038F000174DA84203D005F50065A84206D123F470
:103900000043CD6843EA053323F48043104DA842B9
:103910000FD005F50065A8420BD005F54065A8421B
:1039200007D005F58065A84203D005F58065A8425B
:1039300007D124F4404C4C694CEA841C8C694CEA55
:1039400084144460C2614A680264036230BC7047F8
:10395000002C014030B4036A026A22F48032026211
:103960004468026D22F4803222F070020D68154323
:1039700023F400338A6843EA02430F4A90420FD08F
:1039800002F5006290420BD002F54062904207D0EF
:1039900002F58062904203D002F58062904204D129
:1039A00024F480344A6944EA0224446005654A6884
:1039B0008264036230BC7047002C014030B4036A5B
:1039C000026A22F4801202624468026D22F0807260
:1039D00022F4E0420D6842EA052223F400138D68C8
:1039E00043EA05530F4DA8420FD005F50065A842E4
:1039F0000BD005F54065A84207D005F58065A842C3
:103A000003D005F58065A84204D124F480244D69D3
:103A100044EA8524446002654A68C264036230BC9B
:103A2000704700BF002C014010B4036A046A24F000
:103A300001040462846924F0F00C4CEA021223F0C1
:103A40000A030B43826103625DF8044B704710B4B4
:103A5000036A046A24F010040462846924F4704C3C
:103A60004CEA023223F0A00343EA011382610362AD
:103A70005DF8044B7047836823F4401323F0700310
:103A80000B4343F0070383607047000090F83D301C
:103A9000012B32D1022380F83D300268D36843F015
:103AA0000103D3600368184A934218D0B3F1804FE2
:103AB00015D0A2F59432934211D002F58062934260
:103AC0000DD002F59632934209D002F5406293423E
:103AD00005D01A6842F001021A6000207047996808
:103AE0000A4A0A40062A0AD0B2F5803F09D01A686D
:103AF00042F001021A600020704701207047002048
:103B000070470020704700BF002C014007000100F3
:103B100070477047704770477047704770B50546EB
:103B20000368DE681C6914F0020F10D016F0020F53
:103B30000DD06FF002021A610123037703689B69BD
:103B400013F0030F7CD0FFF7E6FF00232B7714F070
:103B5000040F12D016F0040F0FD02B686FF0040280
:103B60001A6102232B772B689B6913F4407F6DD079
:103B70002846FFF7D0FF00232B7714F0080F12D050
:103B800016F0080F0FD02B686FF008021A6104239B
:103B90002B772B68DB6913F0030F5ED02846FFF705
:103BA000BAFF00232B7714F0100F12D016F0100F6D
:103BB0000FD02B686FF010021A6108232B772B6847
:103BC000DB6913F4407F4FD02846FFF7A4FF0023A2
:103BD0002B7714F0010F02D016F0010F4BD114F423
:103BE000025F02D016F0800F4DD114F4807F02D016
:103BF00016F0800F4FD114F0400F02D016F0400F96
:103C000051D114F0200F02D016F0200F53D114F42C
:103C1000801F02D016F4801F55D114F4001F02D06B
:103C200016F4001F57D114F4800F02D016F4800F41
:103C300059D114F4000F02D016F4000F5BD170BDFF
:103C4000FFF768FF2846FFF767FF7EE72846FFF784
:103C500061FF2846FFF760FF8DE72846FFF75AFF10
:103C60002846FFF759FF9CE72846FFF753FF2846F1
:103C7000FFF752FFABE72B686FF001021A6128468D
:103C8000FFF747FFABE72B686FF402521A61284633
:103C900000F0DFFBA9E72B686FF480721A612846F9
:103CA00000F0D8FBA7E72B686FF040021A612846A6
:103CB000FFF733FFA5E72B686FF020021A61284653
:103CC00000F0C6FBA3E72B686FF480121A61284648
:103CD00000F0C1FBA1E72B686FF400121A612846BF
:103CE00000F0BAFB9FE72B686FF480021A61284648
:103CF00000F0B3FB9DE72B686FF400021A612846C1
:103D000000F0ACFB9BE700000368304A90420ED005
:103D1000B0F1804F0BD0A2F59432904207D002F55B
:103D20008062904203D002F59632904203D123F094
:103D300070034A681343254A90421AD0B0F1804F6D
:103D400017D0A2F59432904213D002F580629042CF
:103D50000FD002F5963290420BD002F540629042AD
:103D600007D002F58062904203D002F58062904253
:103D700003D123F44073CA68134323F080034A69D4
:103D8000134303608B68C3620B6883620F4B9842D6
:103D90000FD003F5006398420BD003F540639842BF
:103DA00007D003F58063984203D003F580639842FF
:103DB00001D10B69036301234361036913F0010F10
:103DC00003D0036923F0010303617047002C014015
:103DD00060B310B5044690F83D3013B3022384F865
:103DE0003D30214651F8040BFFF78EFF012384F884
:103DF000483084F83E3084F83F3084F8403084F80E
:103E0000413084F8423084F8433084F8443084F8F8
:103E1000453084F8463084F8473084F83D3000203F
:103E200010BD80F83C30FDF727F8D7E70120704738
:103E300060B310B5044690F83D3013B3022384F804
:103E40003D30214651F8040BFFF75EFF012384F853
:103E5000483084F83E3084F83F3084F8403084F8AD
:103E6000413084F8423084F8433084F8443084F898
:103E7000453084F8463084F8473084F83D300020DF
:103E800010BD80F83C30FFF743FED7E701207047B4
:103E900030B4036A026A22F0100202624468826946
:103EA00022F0807222F4E6420D6842EA052223F0F5
:103EB00020038D6843EA0513174DA84203D005F58A
:103EC0000065A84206D123F08003CD6843EA0513BC
:103ED00023F04003104DA8420FD005F50065A8421D
:103EE0000BD005F54065A84207D005F58065A842CE
:103EF00003D005F58065A84207D124F4406C4C69D5
:103F00004CEA840C8C694CEA8404446082614A68FF
:103F10008263036230BC7047002C014038B590F8D2
:103F20003C30012B00F0958004460D46012380F8BB
:103F30003C30142A00F28880DFE802F00B86868687
:103F40001F86868634868686488686865D86868631
:103F500071000068FFF724FC2268936943F00803AE
:103F600093612268936923F0040393612268936943
:103F700029690B439361002067E00068FFF788FF21
:103F80002268936943F4006393612268936923F480
:103F90008063936122689369296943EA01239361ED
:103FA000002052E00068FFF749FC2268D36943F023
:103FB0000803D3612268D36923F00403D361226824
:103FC000D36929690B43D36100203EE00068FFF705
:103FD0007BFC2268D36943F40063D3612268D36910
:103FE00023F48063D3612268D369296943EA0123FA
:103FF000D361002029E00068FFF7ACFC2268136D54
:1040000043F0080313652268136D23F0040313655E
:104010002268136D29690B431365002015E00068C1
:10402000FFF7CCFC2268136D43F40063136522682C
:10403000136D23F4806313652268136D296943EAC5
:1040400001231365002000E00120002384F83C30A8
:1040500038BD0220FCE710B4846824F47F4C42EAA7
:1040600003220A4342EA0C0282605DF8044B704767
:1040700090F83C30012B00F08F8010B504460123EE
:1040800080F83C30022380F83D3002689068434B52
:10409000034093600B68702B55D031D8502B6CD0F7
:1040A0001FD8402B0AD1CA6849682068FFF7BCFCBA
:1040B00040212068FFF7DFFC002029E068D8202B92
:1040C00003D00AD80BB1102B05D119462068FFF791
:1040D000D2FC00201CE001201AE0302BF5D001209A
:1040E00016E0602B0AD1CA6849682068FFF7AFFC68
:1040F00060212068FFF7BFFC002009E0012007E0F5
:10410000B3F5005F2CD00AD8B3F5805F42D1002010
:10411000012384F83D30002384F83C3010BD204A50
:104120009342D2D007D8B3F1101FCED0103A9342A9
:10413000CBD00120ECE71B4A9342C6D030329342E9
:10414000C3D00120E4E7CB684A6889682068FFF79C
:1041500082FF2268936843F0770393600020D7E7DB
:10416000CB684A6889682068FFF775FF2268936802
:1041700043F4804393600020CAE7CA684968206816
:10418000FFF752FC50212068FFF775FC0020BFE7C5
:104190000120BDE70120BBE7022070478800CEFF69
:1041A000300010004000100001F01F014FF0010C22
:1041B0000CFA01FC036A23EA0C030362036A8A40D7
:1041C000134303627047000010B50446102928D835
:1041D000DFE801F0092727270F272727152727279B
:1041E0001B272727210090F83E30013B18BF0123F1
:1041F0001CE090F83F30013B18BF012316E090F817
:104200004030013B18BF012310E090F84130013BE2
:1042100018BF01230AE090F84230013B18BF012388
:1042200004E090F84330013B18BF0123002B6AD112
:1042300010291ED8DFE801F0091D1D1D0D1D1D1DD3
:10424000111D1D1D151D1D1D1900022384F83E3072
:1042500012E0022384F83F300EE0022384F840305D
:104260000AE0022384F8413006E0022384F8423059
:1042700002E0022384F8433001222068FFF794FF14
:104280002368244A93420FD002F5006293420BD078
:1042900002F54062934207D002F58062934203D058
:1042A00002F58062934203D15A6C42F400425A6490
:1042B0002368184A934218D0B3F1804F15D0A2F565
:1042C0009432934211D002F5806293420DD002F5F0
:1042D0009632934209D002F54062934205D01A68A3
:1042E00042F001021A6000200EE099680A4A0A4072
:1042F000062A0AD0B2F5803F09D01A6842F00102BE
:104300001A60002000E0012010BD0020FCE7002022
:10431000FAE700BF002C01400700010090F83C20A4
:10432000012A40D030B40346012280F83C2002220A
:1043300080F83D200068426884681C4DA84203D084
:1043400005F50065A84203D122F470024D682A43A6
:1043500022F0007222F070020D682A4342601A684F
:104360001248824212D0B2F1804F0FD0A0F59430A3
:1043700082420BD000F58060824207D000F5963073
:10438000824203D000F54060824204D124F08004D0
:10439000896821439160012283F83D20002083F841
:1043A0003C0030BC70470220704700BF002C014029
:1043B00090F83C30012B46D010B40246012380F81F
:1043C0003C30CB6823F440738868034323F4806354
:1043D0004868034323F400630868034323F48053CD
:1043E0000869034323F400534869034323F48043DB
:1043F000086B034323F47023886943EA004323F0E6
:104400008053C86903431068104CA04203D004F5E0
:104410000064A04210D123F470038C6A43EA045371
:1044200023F080730C6A234323F000734C6A234308
:1044300023F00053C96A0B434364002082F83C0018
:104440005DF8044B70470220704700BF002C01400C
:1044500070477047704770477047704770470268F1
:1044600052E8003F23F0C00342E800310029F6D1B2
:10447000026802F1080353E8003F23F40003083206
:1044800042E800310029F3D12023C0F8883070477A
:10449000026852E8003F23F4907342E8003100299B
:1044A000F6D1026802F1080353E8003F23F080537D
:1044B00023F00103083242E800310029F1D1C36E34
:1044C000012B06D02023C0F88C300023C36643673D
:1044D0007047026852E8003F23F0100342E80031C1
:1044E0000029F6D1EEE700001346D0F88820202AF4
:1044F0003DD110B5044600293BD0002B3BD00165CF
:10450000A0F85430A0F856300022C0F890202122A4
:10451000C0F88820C26FCAB11849D162C26F184969
:104520001163C26F17495163C26F00219163026822
:104530002832016DC06FFDF75BFD38B11023C4F860
:1045400090302023C4F8883001200FE023684022F7
:104550001A62226802F1080353E8003F43F0800327
:10456000083242E800310029F3D1002010BD0220BA
:1045700070470120FAE70120F8E700BF89450008ED
:10458000F54500080146000808B50346806A1B6827
:104590001B6813F0200F18D10023A0F856300268D2
:1045A00002F1080353E8003F23F08003083242E899
:1045B00000310029F3D1026852E8003F43F0400384
:1045C00042E800310029F6D108BDFBF757FFFBE7B1
:1045D00008B5026852E8003F23F0400342E800318A
:1045E0000029F6D12023C0F8883000238367FBF729
:1045F00045FF08BD08B5806AFBF746FF08BD704758
:1046000038B5846AD4F88820D4F88C5023689B6825
:1046100013F0800F01D0212A10D023689B6813F07B
:10462000400F01D0222D10D0D4F8903043F0100369
:10463000C4F890302046FFF7E2FF38BD0023A4F80D
:1046400056302046FFF70BFFE7E70023A4F85E3063
:104650002046FFF71DFFE7E708B5806A0023A0F8B2
:104660005E30FFF7CCFF08BD70B504460268D36921
:104670001068916840F60F0C13EA0C0F0DD113F07F
:10468000200F10D010F0200F02D111F0805F0AD05F
:10469000636F93B3204698472FE09D4D0D402DD179
:1046A0009C4E30422AD1E56E012D00F0C08013F4FB
:1046B000801F03D011F4800F40F06C8113F0800F45
:1046C00007D010F0800F40F06C8111F4000F40F023
:1046D000688113F0400F03D010F0400F40F0688164
:1046E00013F4000F03D010F0804F40F0658113F0F9
:1046F000807F02D00028C0F2638170BD13F0010FEB
:1047000009D010F4807F06D001261662D4F89020DC
:104710003243C4F8902013F0020F0BD011F0010FB8
:1047200008D0226802261662D4F8902042F00402D3
:10473000C4F8902013F0040F0BD011F0010F08D033
:10474000226804261662D4F8902042F00202C4F8CF
:10475000902013F0080F0BD010F0200F00D13DB1C6
:10476000226808251562D4F890202A43C4F89020C6
:1047700013F4006F0CD010F0806F09D022684FF452
:1047800000651562D4F8902042F02002C4F8902011
:10479000D4F89020002AB0D013F0200F09D010F0E8
:1047A000200F02D111F0805F03D0636F0BB1204660
:1047B0009847D4F8902023689B6813F0400F02D1EB
:1047C00012F0280F2CD02046FFF762FE23689B686A
:1047D00013F0400F20D0226802F1080353E8003F95
:1047E00023F04003083242E800310029F3D1D4F825
:1047F00080306BB1484A9A63D4F88000FDF776FCAC
:1048000000283FF47AAFD4F88000836B984774E7B0
:104810002046FFF7F4FE70E72046FFF7F0FE6CE756
:104820002046FFF7ECFE0023C4F8903065E713F054
:10483000100F3FF43CAF10F0100F3FF438AF1023CF
:10484000136223689B6813F0400F67D0D4F8801080
:104850000A6853689BB2002B4AD0B4F85C009842B7
:1048600046D9A4F85E300B681B6813F0200F32D1D4
:10487000226852E8003F23F4807342E800310029A7
:10488000F6D1226802F1080353E8003F23F0010348
:10489000083242E800310029F3D1226802F108030E
:1048A00053E8003F23F04003083242E8003100297A
:1048B000F3D12023C4F88C300023E366226852E849
:1048C000003F23F0100342E800310029F6D1D4F86C
:1048D0008000FDF7D6FB02232367B4F85C10B4F820
:1048E0005E309BB2C91A89B22046FBF7B3FD04E7DC
:1048F000B4F85C1099427FF400AF136813F0200FF6
:104900003FF4FBAE022323672046FBF7A3FDF4E64A
:10491000010000102001000459460008B4F85C10A2
:10492000B4F85E309BB2C91A89B2B4F85E309BB25B
:10493000002B3FF4E2AE00293FF4DFAE226852E8DC
:10494000003F23F4907342E800300028F6D122683B
:1049500002F1080353E8003F23F0805323F00103E2
:10496000083242E800300028F1D12023C4F88C300E
:104970000023E3666367226852E8003F23F01003D8
:1049800042E800300028F6D1022323672046FBF7D7
:1049900061FDB2E64FF480131362204600F022FB63
:1049A000ABE6A36F002B3FF4A8AE20469847A4E6E1
:1049B0002046FFF70DFEA0E6204600F015FB9CE622
:1049C000204600F010FB98E670B504468368026943
:1049D000134342691343C2691343016808688A4A52
:1049E00002401A430A602268536823F44053E16886
:1049F0000B435360A1692268844B9A4201D0236A19
:104A00001943936823F06E4323F430630B439360A0
:104A10002268D36A23F00F03616A0B43D3622368D1
:104A20007B4A934223D07B4A934234D07A4A9342C2
:104A30004AD07A4A934259D0744A934268D010229D
:104A400072498B4200F09580E069B0F5004F00F0AC
:104A5000D080082A00F24281DFE812F0100129011B
:104A60000E0140012C014001400140012F0102F5DF
:104A70005842D2F8882002F00302032A09D8DFE85E
:104A800002F002045C060122DAE70422D8E70822D9
:104A9000D6E71022D4E702F5E632D2F8882002F0F9
:104AA0000C020C2A0ED8DFE802F0070D0D0D090DDF
:104AB0000D0D4A0D0D0D0B000022C1E70422BFE7CA
:104AC0000822BDE71022BBE702F5E432D2F88820C5
:104AD00002F03002202A34D004D8A2B3102A34D1F4
:104AE0000422ADE7302A32D10822A9E702F5E232EA
:104AF000D2F8882002F0C002802A2AD004D852B30B
:104B0000402A2AD104229BE7C02A28D1082297E70D
:104B100002F5C832D2F8882002F44062B2F5006F84
:104B20001FD005D8FAB1B2F5806F1ED1042287E7F5
:104B3000B2F5406F1BD1082282E7022280E70222F1
:104B40007EE702227CE700227AE7102278E7102233
:104B500076E7022274E7002272E7102270E7102243
:104B60006EE702226CE700226AE7102268E7102253
:104B700066E7082A00F2A480DFE802F008A210A28B
:104B80000DA2A2A205004FF4004008E0FCF7E0FEF1
:104B900028B90020A3E0FCF795FDF9E72048626AF8
:104BA000204B33F81220B0FBF2F3656805EB4501AA
:104BB000994200F28780B3EB053F00F28580002622
:104BC00033463146FBF75CFB090241EA1061000203
:104BD0006B08C0182A46334641F10001FBF750FB31
:104BE000A0F54072104B9A4270D82368D8603046C6
:104BF00075E0082A6CD8DFE802F01939056B3C6BC8
:104C00006B6B1D00064815E0F369FFCF0080004084
:104C1000003801400044004000480040004C004083
:104C20000024F4006C620008FFFC0F00FCF790FE0B
:104C300000284FD0626A304B33F81230B0FBF3F0EB
:104C40006268530803EB4003B3FBF2F3A3F11001D6
:104C50004FF6EF7291423FD89AB222F00F02C3F39F
:104C6000420313432268D360002038E0FCF782FE41
:104C7000DEE7FCF727FDDBE7204802E0FCF768FEF3
:104C8000B0B3626A1C4B33F81230B0FBF3F06368C8
:104C900000EB5300B0FBF3F0A0F110024FF6EF73FE
:104CA0009A4227D8236880B2D860002017E0FCF72A
:104CB00061FEE5E7FCF706FDE2E74FF40040E0E7C0
:104CC00001200CE001200AE0012008E0012006E0BC
:104CD000012004E0002002E0012000E00120012387
:104CE000A4F86A30A4F8683000236367A36770BD36
:104CF0000020F4E70120F2E76C6200080024F400D1
:104D0000836A13F0080F06D00268536823F4004347
:104D1000816B0B435360836A13F0010F06D0026866
:104D2000536823F40033C16A0B435360836A13F062
:104D3000020F06D00268536823F48033016B0B43E3
:104D40005360836A13F0040F06D00268536823F49B
:104D50008023416B0B435360836A13F0100F06D01E
:104D60000268936823F48053C16B0B439360836A9A
:104D700013F0200F06D00268936823F40053016CEF
:104D80000B439360836A13F0400F0AD002685368A4
:104D900023F48013416C0B435360436CB3F5801FC5
:104DA0000BD0836A13F0800F06D00268536823F497
:104DB0000023C16C0B43536070470268536823F4AF
:104DC000C003816C0B435360EBE72DE9F8430546C4
:104DD0000E4617469946DDF820802B68DC6936EAD6
:104DE00004040CBF01240024BC4236D1B8F1FF3FBB
:104DF000F3D0FCF795F9A0EB0900404530D8B8F1A5
:104E0000000F2FD02B681A6812F0040FE5D0802E07
:104E1000E3D0402EE1D0DA6912F0080F11D1DA693F
:104E200012F4006FD9D04FF400621A622846FFF7DF
:104E30002FFB2023C5F89030002385F88430032011
:104E40000CE008241C622846FFF722FBC5F89040BE
:104E5000002385F88430012000E00020BDE8F883BD
:104E60000320FBE70320F9E730B583B004460023B5
:104E7000C0F89030FCF754F905462268126812F029
:104E8000080F10D123681B6813F0040F28D12023CA
:104E9000C4F88830C4F88C300020E066206784F8BD
:104EA000840003B030BD6FF07E43009303460022C0
:104EB0004FF400112046FFF788FF0028E2D0226857
:104EC00052E8003F23F0800342E800310029F6D188
:104ED0002023C4F88830002384F884300320E0E7DE
:104EE0006FF07E4300932B4600224FF48001204652
:104EF000FFF76BFF0028CAD0226852E8003F23F476
:104F0000907342E800310029F6D1226802F10803CB
:104F100053E8003F23F00103083242E80031002942
:104F2000F3D12023C4F88C30002384F8843003208C
:104F3000B7E778B310B50446D0F888300BB3242314
:104F4000C4F888302268136823F001031360A36A51
:104F5000E3B92046FFF738FD012811D022685368D5
:104F600023F4904353602268936823F02A039360EC
:104F70002268136843F0010313602046FFF774FFB3
:104F800010BD80F88430FCF703F8D8E72046FFF71F
:104F9000B7FEDEE701207047436E2BB90123A0F86E
:104FA0006A30A0F86830704730B403689A68C2F37A
:104FB00042629968490F094D6B5CDB00084C615CEB
:104FC00093FBF1F3A0F86A30AB5CDB00A25C93FBCF
:104FD000F2F3A0F8683030BC704700BF8C62000864
:104FE0008462000870477047704790F88430012B46
:104FF00018D0012380F884302423C0F88830036857
:105000001A68196821F00101196022F0005200238A
:10501000436601680A602022C0F8882080F8843046
:10502000184670470220704738B590F88430012B3D
:105030001DD00446012380F884302423C0F8883032
:1050400003681D681A6822F001021A6002689368FA
:1050500023F0604319439160FFF79EFF23681D60B2
:105060002023C4F88830002084F8840038BD022052
:10507000FCE738B590F88430012B1DD0044601239D
:1050800080F884302423C0F8883003681D681A68CB
:1050900022F001021A600268936823F060631943EA
:1050A0009160FFF779FF23681D602023C4F88830E2
:1050B000002084F8840038BD0220FCE7034AD2F8BF
:1050C000883043F47003C2F88830704700ED00E088
:1050D00010B503460C4A0D490D48006840B10C4814
:1050E00000680344521A934206D8094A136010BD5F
:1050F0000748084C0460F2E700F0B4FA0C230360A0
:105100004FF0FF30F3E700BF0080002000040000F4
:1051100048040020C006002010B50C468AB20146A3
:105120000348FFF7E1F9034B00221A70204610BD37
:105130003C01002064040020064B074A1A6000234B
:10514000064A1370064A136053609360D360054AA1
:10515000137070476004002098BC14004E040020B7
:10516000500400204D040020114B1B78FBB942680D
:1051700040F618439A4204D901230E4A13700C4A90
:105180001370826840F618439A4205D9094B0322EE
:105190001A70074B01221A70C26840F618439A42EF
:1051A00005D9044B02221A70014B01221A70704774
:1051B0004E0400204D04002008B5114B1B7813B19C
:1051C000104A127822B113B90E4B1B784BB908BDA7
:1051D0000D49452000F078F8094B1A78094B1A70F0
:1051E000F5E70A49492000F06FF80020084B1870D5
:1051F00000F08AF8024B1A78024B1A70E7E700BFFA
:105200004E0400204C040020AC620008B462000888
:105210004D04002038B5234C2078234D234B1B68C8
:10522000234A4FF48071284400F0DEF923781844B3
:10523000C0B220704FF4FF631E4A4FF480712844BF
:1052400000F0D2F920780930C0B2207040F618433F
:10525000194A4FF48071284400F0C6F920780830CC
:10526000C0B2207040F61843144A4FF480712844AD
:1052700000F0BAF920780830C0B2207040F6184328
:105280000F4A4FF48071284400F0AEF923780833B8
:10529000DBB223700B4A1288EA52DBB2013323706F
:1052A00038BD00BF640400206804002060040020B2
:1052B000BC620008C8620008D0620008D86200081A
:1052C000E0620008E862000810B582B00346074CAF
:1052D00094F800C00091064A4FF48071054860447C
:1052E00000F082F9207002B010BD00BF64040020FD
:1052F000EC6200086804002008B502494920FFF765
:10530000E3FF08BDF862000808B5002851D0024646
:105310002B4B1B7813B92B49098869B11BB9294953
:105320000988092911D8012B1BD0022B37D0254A17
:1053300013880133138041E0012210212248FCF739
:105340008EFD204B01221A8038E0002210211E48D9
:10535000FCF785FD1A4B01221A701A4B00221A80A5
:105360002CE0184909880929DFD9184B1B78013A24
:10537000934209DA0133154A1370114B00221A7057
:10538000104B00221A8019E00D4B02221A700022E5
:105390000E4B1A7010210C48FCF761FDF0E7094B29
:1053A0001B884F2BC3D90023054A1370054A13806D
:1053B00004E0002210210448FCF751FD08BD00BFA5
:1053C0007205002070050020000400486E050020D2
:1053D000014BD863704700BF0034014010B5B0F5F1
:1053E000006F17D3A0F50064A4B2B4F5FF6F16D810
:1053F000164B1B8842F20F72934219D80133134A9D
:105400001380134B1B88A3421BD8114B1C80104BDD
:10541000188810BDC0F5FF640734A4B2E5E70B4B54
:1054200000221A80012240210A48FCF718FDE8E713
:10543000002240210748FCF712FD044B00221A808D
:10544000DFE7013B024A1380E1E700BF6C05002063
:105450006A0500200004004800B5A2EB010C1FFA09
:105460008CFCBDF804E0AEEB030E1FFA8EFEBCFB15
:10547000FEFC07EE90CAB8EEE77A824294BFC1EB19
:105480000201C1EB000107EE901AF8EEE77AC7EED1
:10549000876A07EE903AF8EEE77A77EEA67AFCEEA6
:1054A000E77A17EE903A98B25DF804FB2DE9F041E7
:1054B00082B06427009700234FF4006219462C48FD
:1054C0000088FFF7C9FF03462A4C20782A4E2B4A52
:1054D0004FF48071304400F087F825780544EDB230
:1054E0002570DFF8AC800097002340F6FF72194664
:1054F000B8F80400FFF7B0FF0346214A4FF480716B
:10550000701900F071F825780544EDB22570009708
:10551000002340F6FF721946B8F80800FFF79CFF19
:105520000346184A4FF48071701900F05DF8257831
:105530000544EDB225700097002340F6FF7219462E
:10554000B8F80C00FFF788FF03460F4A4FF480714C
:10555000701900F049F823781844C0B220700B4B42
:105560001B883352C3B20133237002B0BDE8F0810F
:10557000740500206404002068040020086300080B
:10558000146300081C63000824630008E862000834
:10559000500400200D488546FFF790FD0C480D494A
:1055A0000D4A002302E0D458C4500433C4188C427E
:1055B000F9D30A4A0A4C002301E013600432A242E4
:1055C000FBD300F055F8FBF70BFAFEE70080002054
:1055D000000000205C000020706300085C000020D8
:1055E000C0060020FEE700000CB430B5184B0C1EBE
:1055F0001D689DB008DA8B232B604FF0FF301DB083
:10560000BDE8304002B070474FF40273ADF814307B
:105610004FF000031B9314BF04F1FF3323460493A0
:1056200007934FF6FF7302900690ADF81630209A5C
:1056300021AB02A92846019300F0A6F9431CBCBF88
:105640008B232B60002CDAD0029B00221A70D6E745
:105650000C00002002440346934200D1704703F837
:10566000011BF9E7014B1868704700BF0C000020D0
:1056700070B50D4B0D4D5B1B9C100026A64209D149
:1056800000F0E8FD0A4D0B4B5B1B9C100026A64268
:1056900005D170BD55F8043B98470136EEE755F843
:1056A000043B98470136F2E7686300086863000826
:1056B000686300086C630008704770470A449142B1
:1056C00000F1FF3300D1704710B511F8014B03F81A
:1056D000014F9142F9D110BD38B50546002941D09E
:1056E00051F8043C0C1F002BB8BFE41800F0E0F8A0
:1056F0001D4A136833B9636014602846BDE838401A
:1057000000F0DCB8A34208D9206821188B4201BF01
:1057100019685B6809182160EDE71A465B680BB1F0
:10572000A342FAD911685018A0420BD12068014455
:10573000501883421160E0D118685B6853600844D8
:105740001060DAE702D90C232B60D6E72068211815
:105750008B4204BF19685B68636004BF091821604D
:105760005460CAE738BD00BFBC06002070B50F4EBC
:105770000C463168054611B900F0AAFB306021469D
:10578000284600F0A5FB431C03D14FF0FF34204610
:1057900070BDC41C24F00304A042F8D0211A28468E
:1057A00000F096FB0130F2D1EFE700BFB806002011
:1057B0002DE9F843CD1C25F0030508350C2D38BF25
:1057C0000C25002D064601DBA94204D90C233360C9
:1057D0000020BDE8F883DFF8D48000F069F8D8F83D
:1057E00000301C4644BB29463046FFF7BFFF431C30
:1057F000044658D1D8F800402746002F43D1002C4A
:105800004BD023683946304604EB030900F060FBB7
:10581000814542D121686D1A29463046FFF7A6FF1F
:1058200001303AD023682B442360D8F800305A68FE
:1058300062BBC8F800700FE02268521B20D40B2A0C
:1058400017D96119A342256018BF5960636808BF62
:10585000C8F8001062514B60304600F02FF804F198
:105860000B00231D20F00700C21A1CBF1B1AA350F7
:10587000AFE76268A3420CBFC8F800205A60EBE7AC
:1058800023466468AEE73C467F68B6E71A465B6825
:10589000A342FBD100235360DEE70C233360304684
:1058A00000F00CF894E70560D6E700BFBC060020C6
:1058B0000148FFF701BF00BFB40600200148FFF711
:1058C000FCBE00BFB40600202DE9F0478E681F46DD
:1058D000BE4282460C469046334653D8B1F90C007E
:1058E00010F4906F2BD065692368096905EB4505B5
:1058F000A3EB010905EBD5757B1C6D104B44AB4246
:105900002A4684BF1D462A46430527D511465046E0
:10591000FFF74EFF064658B321694A46FFF7CEFE11
:10592000A38923F4906343F08003A381266165611A
:105930004E44A5EB09052660A5603E463B461F4642
:1059400020683A46414600F0A9FAA3689B1BA36071
:1059500023683B4423600020BDE8F087504600F0F8
:10596000C7FA06460028E1D121695046FFF7B4FE88
:105970000C23CAF80030A38943F04003A3814FF001
:10598000FF30E9E73E46DBE72DE9F04F98468B898B
:105990001B069DB007460D46144610D50B6973B91A
:1059A0004021FFF705FF2860286130B90C233B60D8
:1059B0004FF0FF301DB0BDE8F08F40236B61002336
:1059C000099320238DF82930CDF80C803023DFF89F
:1059D0009C818DF82A304FF0010923469A4613F82E
:1059E000012B0AB1252AF9D1BAEB040B0BD05B4687
:1059F000224629463846FFF767FF013000F0A780AE
:105A0000099A5A4409929AF80030002B00F09F80BE
:105A100000234FF0FF32CDE905230AF1010A049378
:105A200007938DF853301A935446052214F8011B3E
:105A30004E48FAF7D5FB049AD8B9D00644BF2023C4
:105A40008DF85330110744BF2B238DF853309AF84B
:105A500000302A2B15D0079A544600204FF00A0C2C
:105A6000214611F8013B303B092B4BD9B0B10792CD
:105A700014E0A0EB080309FA03F313430493A246CE
:105A8000D2E7039B191D1B680391002BBBBF5B4230
:105A900042F0020207930793B8BF049223782E2B9B
:105AA0000AD163782A2B32D1039B1A1D1B680392FB
:105AB00043EAE37302340593DFF8C0A021780322A0
:105AC0005046FAF78DFB38B1049BA0EB0A00402248
:105AD000824013430134049314F8011B24488DF8C9
:105AE00028100622FAF77CFB002836D0214B1BBB7E
:105AF000039B073323F0070308330393099B3344C5
:105B000009936AE70CFB02320C460120A8E7002348
:105B10000134059319464FF00A0C204610F8012B6A
:105B2000303A092A03D9002BC6D00591C4E70CFBF3
:105B3000012104460123F0E703AB00932A460E4BF4
:105B400004A93846AFF30080421C0646D6D1AB8983
:105B50005B063FF52DAF09982CE703AB00932A466F
:105B6000054B04A9384600F079F8EDE72A630008F0
:105B70003463000800000000C958000830630008C2
:105B80002DE9F047164698468A680B69DDF82090A3
:105B90009342B8BF1346336091F8432007460C4642
:105BA0000AB1013333602368990642BF3368023378
:105BB0003360256815F0060506D104F1190AE3687B
:105BC00032689B1AAB4226DC94F843302268003BD3
:105BD00018BF012392062BD404F1430241463846F4
:105BE000C84701301ED02368226903F00603042B46
:105BF00002BFE5683368ED1AA3680CBF25EAE575B6
:105C000000259342C4BF9B1AED1800261A34B542F2
:105C10001AD1002008E00123524641463846C847C1
:105C2000013003D14FF0FF30BDE8F0870135C6E702
:105C3000E1185A1C302081F84300224494F84510A2
:105C400082F843100233C7E7012322464146384613
:105C5000C8470130E6D00136D9E700002DE9FF47FB
:105C60000F7E0C9E782F914680460C469A4601F195
:105C7000430207D8622F0AD8002F00F0D280582F95
:105C800000F0B78004F1420684F842703AE0A7F1D0
:105C90006303152BF6D801A151F823F0F55C000839
:105CA000095D0008855C0008855C0008855C0008CB
:105CB000855C0008095D0008855C0008855C0008BB
:105CC000855C0008855C0008095E0008335D0008FB
:105CD000BF5D0008855C0008855C00082B5E00083D
:105CE000855C0008335D0008855C0008855C000861
:105CF000C75D000833681A1D1B68326004F1420654
:105D000084F8423001239DE033682068191D31601A
:105D1000060601D51D6803E04506FBD5B3F9005022
:105D2000002D03DA2D236D4284F8433059480A23AD
:105D300010E021683368080653F8045B02D4490672
:105D400048BFADB26F2F5348336059D108230021AB
:105D500084F843106668A660002E05DB21682E4398
:105D600021F0040121604DD01646B5FBF3F103FB91
:105D70001157C75D06F8017D2F46BB420D46F4D989
:105D8000082B0BD12368DF0708D523696168994286
:105D9000DEBF302306F8013C06F1FF36921B22617C
:105DA000CDF800A04B4603AA21464046FFF7E8FE87
:105DB00001304CD14FF0FF3004B0BDE8F0872368CC
:105DC00043F0200323603448782784F84570236823
:105DD00031681F0651F8045B02D45F0648BFADB2BC
:105DE0003160D90744BF43F0200323601DB1102365
:105DF000ADE72848E9E7236823F020032360F6E7AE
:105E00000A23A4E71646BBE7336825686169181DB5
:105E100030602E061B6801D5196002E06806FBD5CC
:105E20001980002323611646BAE733681A1D3260D1
:105E30001E68626800213046FAF7D2F908B1801B6B
:105E4000606063682361002384F84330A8E7236916
:105E5000324649464046D0470130ABD023689B07C5
:105E600013D4E068039B9842B8BF1846A4E7012307
:105E7000324649464046D04701309BD00135E36861
:105E800003995B1AAB42F2DCEBE7002504F119063B
:105E9000F5E700BF3B6300084C630008884210B57B
:105EA00001EB020402D98442234607D8431EA142D3
:105EB00007D011F8012B03F8012FF8E702448242C2
:105EC00000D110BD13F8011D02F8011DF7E7000015
:105ED00038B5064D0023044608462B60FFF7F8F856
:105EE000431C02D12B6803B1236038BDB0060020EB
:105EF0002DE9F041074614460D4621B9BDE8F041B1
:105F00001146FFF755BC2AB9FFF7E6FB25462846A0
:105F1000BDE8F08100F01AF88442064602D8B4EBDE
:105F2000500FF4D821463846FFF742FC804608B9A6
:105F30004546ECE7B4422246294628BF3246FFF7E1
:105F4000BDFB29463846FFF7C7FBF1E751F8043C93
:105F5000181F002BBCBF0B58C01870472DE9F04725
:105F6000089D0F4604468C46002B48D18A421646AF
:105F700061D9B2FA82F34BB1C3F1200201FA03FCFA
:105F800020FA02F29E4042EA0C0C9C404FEA164E68
:105F9000B7B2BCFBFEF1220C0EFB11CC42EA0C4264
:105FA00001FB07F0904209D9B21801F1FF3C80F0E3
:105FB000EE80904240F2EB8002393244121AA4B2D1
:105FC000B2FBFEF00EFB102244EA024400FB07F78E
:105FD000A74209D9341900F1FF3280F0DA80A742D4
:105FE00040F2D7803444023840EA0140E41B0021EB
:105FF0001DB1DC400023C5E90043BDE8F0878B42BA
:1060000006D90DB1C5E9000100210846BDE8F087B9
:10601000B3FA83F1002948D1BB4202D3824200F295
:106020000781841A67EB030201209446002DE4D017
:10603000C5E9004CE1E7002A00F09280B2FA82F351
:10604000002B40F0A8808A1A4FEA164E1FFA86FCF1
:106050000121200CB2FBFEF70EFB172240EA0242A0
:106060000CFB07F0904207D9B21807F1FF3802D2B3
:10607000904200F2E2804746121AA4B2B2FBFEF050
:106080000EFB102244EA02440CFB00FCA44507D995
:10609000341900F1FF3202D2A44500F2CB80104641
:1060A000A4EB0C0440EA0740A2E7C1F120068B40B4
:1060B00022FA06FC4CEA030C07FA01F420FA06F374
:1060C000F7404FEA1C49234300FA01F81FFA8CFEFF
:1060D000B7FBF9F01C0C09FB107744EA074400FBFE
:1060E0000EF7A74202FA01F20AD91CEB040400F1F0
:1060F000FF3A80F09B80A74240F2988002386444C7
:10610000E41B9FB2B4FBF9F309FB134447EA0444D0
:1061100003FB0EFEA64509D91CEB040403F1FF376F
:1061200080F08280A6457FD9023B644443EA004068
:10613000A4EB0E04A0FB02E7BC427346B94663D34E
:1061400060D05DB1B8EB030264EB090404FA06F613
:1061500022FA01F31E43CC40C5E9006400214CE75C
:106160006208480842EAC1710B0C43EA00438AB254
:1061700042EA0342B3FBF6F1E407B4463746B646BB
:106180001F23B0FBF6F0D21B41EA004161E76146F4
:1061900014E7104628E7C3F1200120FA01F29E40DF
:1061A00027FA01F19F403A434FEA164E1FFA86FC48
:1061B000B1FBFEF70EFB1710110C41EA004107FB83
:1061C0000CF8884504FA03F43AD9711807F1FF3046
:1061D00001D288451FD8A1EB0801B1FBFEF808FBEE
:1061E0000CF70EFB181192B242EA0142BA422FD2CA
:1061F000B21808F1FF31C6D2BA42C4D2A8F10201E6
:106200003244C0E7F0459CD2BEEB020367EB0C07BB
:106210000138B94695E7A6EB08084144B81EB1FB22
:10622000FEF808FB0CF7DCE73B467FE7504667E7E4
:106230000846FBE63444023832E7023F32441BE7AB
:10624000A1EB08013846B1FBFEF808FB0CF7C8E7E4
:10625000414698E7F8B500BFF8BC08BC9E467047B9
:0C626000F8B500BFF8BC08BC9E467047B3
:10626C00010002000400060008000A000C001000E7
:10627C002000400080000001080402040801010114
:10628C0001010103070100000000000001020304EA
:10629C0000000000000000000102030406070809CA
:1062AC004C4F434B21000000554E4C4F434B0000CC
:1062BC00444D5020463D256C7520000056504B3DFA
:1062CC002575200053543D257520000053443D2571
:1062DC007520000053523D25752000000A00000077
:1062EC004C4F472025632025730A000073657269A3
:1062FC006F7720554920696E69740000444D502019
:10630C00563D257520000000543D257520000000E9
:10631C00443D257520000000523D25752000232D9D
:10632C00302B2000686C4C00656667454647003092
:10633C0031323334353637383941424344454600DF
:10634C0030313233343536373839616263646566DF
:04635C00000000003D
:08636000809EFF7F0100000098
:046368001D03000809
:04636C00F50200082E
:1063700001000000100000000024F40010000020C4
:106380000000000078050020E005002048060020FD
:1063900000000000000000000000000000000000FD
:1063A00000000000000000000000000000000000ED
:1063B00000000000000000000000000000000000DD
:0C63C000000000000000000000000000D1
:040000050800559505
:00000001FF
